:040000008A11222C13
:10060000FE00FE1F082B83137E18831700080800C6
:100610000408FE0003308A007E08820700344F344D
:100620004B343E3400347E088A007F088200132356
:100630008A118000840A04087D0603190034FF0A29
:100640000319FE0A172B01308312031386008A1147
:10065000C4248A110A308A1108248A11080064000F
:0E0660008001840A0406031900340406302BBE
:10078A0083120313D200520886008A119D248A110B
:10079A000D3083120313D3000130D302031DD62B6D
:1007AA00D72BD12B0800F700E52B77088A110923EC
:1007BA008A118A11C5238A110130F6007608F707D3
:1007CA0077088A1109238A110038031DED2BEE2BB5
:1007DA00DA2B080083120313D00003100030031829
:1007EA000130CF003A3050020318FC2BFD2B062CA7
:1007FA0030305002031C022C032C062CCF010314A8
:10080A00CF0D4F0C080083120313CF000430D10020
:10081A005330D0000130D002031D142C152C0F2C9C
:10082A000130D102031D1A2C1B2C0D2C0130CF02D2
:10083A00031D202C212C0B2C0800F001F101F201E0
:10084A00F301F4018313403084004F308A112F23BF
:10085A008A114030FD000430FE005730FF0020307E
:10086A0084008A1117238A1183018A11752F831232
:10087A000313D0000310003003180130CF00501CBE
:10088A00472C482C4C2C7608F5007508CF07031026
:10089A00F60D0310D00CD008031D542C552C442CF3
:1008AA004F08080030343134323433343434353478
:1008BA0036343734383439344134423443344434A6
:1008CA0045344634EE34ED34EB34E734DE34DD348B
:1008DA00DB34D734BE34BD34BB34B7347E347D34D4
:1008EA007B3477340310003003180130F3007308A7
:1008FA00303E8400831300087006031D852C862C65
:10090A008B2C7308203E84000008F2007308013E15
:10091A00F30010307302031C932C942C7C2C720865
:10092A0083120313860064308A1108248A1108008E
:10093A00F11471088312031385001130D1000130BC
:10094A00D102031DA92CAA2CA42C711571088500AB
:10095A001130D0000130D002031DB42CB52CAF2CBD
:10096A00FB30F5007508F105710885001130CF00DC
:10097A000130CF02031DC22CC32CBD2C0800FD3050
:10098A00F5007508F105710883120313850011300B
:10099A00D1000130D102031DD32CD42CCE2C7115D9
:1009AA00710885001130D0000130D002031DDE2C01
:1009BA00DF2CD92CFB30F5007508F105710885008C
:1009CA001130CF000130CF02031DEC2CED2CE72CA7
:1009DA000800003083120313CF000030D000511CEE
:1009EA00F72CF82CFE2C5308CF070318D00A54080A
:1009FA00D00701300310D30DD40DFF3E031DFF2C89
:100A0A0001300310D20CD10CFF3E031D062D5208F3
:100A1A005104031D112D122DF42C5008D201D207B6
:100A2A004F08D101D1070800F0308316031386005E
:100A3A00831203130608C3004308F039C200700882
:100A4A000F39F00070084204F0000608C30043089A
:100A5A00F039C2004208F03A0319342D352D362DEB
:100A6A002A2D031000300318013083160313860061
:100A7A008A1177248A11720883120313C500C401EC
:100A8A000314C40D08000310003003180130F400E9
:100A9A008A11B7258A1183120313C1004108F8008D
:100AAA007408463E84007808831380007408463E22
:100ABA0084000008463A031D632D642D652D732DAD
:100ACA0041088A11C5238A110130F8007808F40711
:100ADA0007307402031C722D732D4D2D03107408F8
:100AEA00463E84000030031801308313800008005A
:100AFA0083120313D300023086008A11C4248A1198
:100B0A000A308A1108248A112830F6008312031346
:100B1A0053088A113C248A11F700831203135408DC
:100B2A007707D3000310003003180130D400B02D2A
:100B3A00143086008A11C4248A11213083120313C7
:100B4A00D2000130D202031DAB2DAC2DA62D0130EF
:100B5A00F7007708D40753085402031CB52DB62DA5
:100B6A009D2D08000310003003180130831203136F
:100B7A00C4000310003003180130831603138500E4
:100B8A00F0308600811303100030031801308312FD
:100B9A0003138500EF30F000700886000430C000AF
:100BAA00112E7008F600F7017608D3007708D400F2
:100BBA000230D5000030D6008A117C268A118313B0
:100BCA00831203135308F000700886000A308A1152
:100BDA0008248A1183120313061EF42DF52D012E03
:100BEA00861EF82DF92D012E061FFC2DFD2D012E36
:100BFA00861B002E012E042E8A1119258A118312B2
:100C0A0003134408013A031D0B2E0C2E0E2E450821
:100C1A00172E4008FF3EC000C008031D152E162ED1
:100C2A00D62DB72D080038308312031386008A1197
:100C3A00C4248A1105308A1108248A113830831293
:100C4A00031386008A11C4248A11213083120313E4
:100C5A00D5000130D502031D332E342E2E2E383006
:100C6A0086008A11C4248A11213083120313D60004
:100C7A000130D602031D422E432E3D2E3830860007
:100C8A008A11C4248A11213083120313D40001303B
:100C9A00D402031D512E522E4C2E013086008A1189
:100CAA00C4248A1132308A1108248A110D30831221
:100CBA00031386008A11C4248A1121308312031374
:100CCA00D2000130D202031D6B2E6C2E662E063026
:100CDA0086008A11C4248A11213083120313D30097
:100CEA000130D302031D7A2E7B2E752E08000310C5
:100CFA0000300318013083120313D000D61F862E4A
:100D0A00872E8F2ED509D609D50A0319D60AD001FE
:100D1A000314D00DD41F922E932E9C2ED309D409DE
:100D2A00D30A0319D40A0130F5007508D006003039
:100D3A00D1000030D200560855040319A52EA62E5C
:100D4A00DE2ECF010314CF0DB52E01300310D50DC1
:100D5A00D60DFF3E031DAB2E0130F5007508CF07F7
:100D6A00D61FB82EB92EAA2E01300310D10DD20DDE
:100D7A00FF3E031DBA2E56085402031DC62E5508FF
:100D8A005302031CC92ECA2ED12E5508D302560867
:100D9A00031CD403D402511401300310D60CD50C11
:100DAA00FF3E031DD22E0130CF02031DDD2EDE2EA3
:100DBA00B92E5008031DE22EE72ED109D209D10A15
:100DCA000319D20A5208D401D4075108D301D30710
:100DDA00080083120313D800F62E0130F5007508B7
:100DEA00D8075808840083130008203A0319FE2EF6
:100DFA00FF2EF22E580884000008093A0319062F1C
:100E0A00072FF22E0030D6000030D7000310003032
:100E1A0003180130D5005808840000082D3A031D34
:100E2A00172F182F212F0130F5007508D50701302B
:100E3A00F5007508D807522F5808840000082B3A85
:100E4A00031D282F292F522F0130F5007508D807C6
:100E5A00522F831203135708D201D2075608D10121
:100E6A00D1070A30D3000030D4008A11EE248A1147
:100E7A008312031358088400831300085107F500EE
:100E8A0052080318520AF6007508D03ED6007608B2
:100E9A000318013EFF3ED700292F58088400000896
:100EAA008A11EF238A1103185B2F5C2F2E2F8312CE
:100EBA0003135508031D622F6E2F5609F5005709B3
:100ECA00F600F50A0319F60A7508D9007608DA0059
:100EDA00742F5708DA01DA075608D901D90708002A
:100EEA0098130730831603139C000310003003186D
:100EFA0001309D0003100030031801309B000310DD
:100F0A000030031801308500031000300318013047
:100F1A0086008312031305108A1118268A118A1172
:100F2A0023238A110310003003180130831203139C
:100F3A00D40000308A117D258A1101308A11D82304
:100F4A008A118A1148258A1146308A11EE268A1199
:100F5A008313831203135A08DC01DC075908DB01E7
:100F6A00DB0715305C06031DBC2F19305B06031D19
:100F7A00BF2FC02FD42F0514FA308A1108248A11E2
:100F8A00FA308A1108248A11FA308A1108248A113F
:100F9A00FA308A1108248A118312031305100330C8
:100FAA005C06031DDA2FF1305B06031DDD2FDE2FF1
:100FBA00942F031000300318013086000F30060208
:100FCA00031CE82FE92FEA2FF52F32308A11082463
:100FDA008A110130F9007908831203138607E32F77
:100FEA00FA308A1108248A11FA308A1108248A11DF
:060FFA00942F8A1100286B
:00000001FF
